:020000040000FA
:100000008B1307309F0083120030850007309F005C
:10001000FF3086008316003086001F308500831273
:10002000A30A05191A28851D262806108614061508
:1000300086111028851921280614861006118615A8
:100040001028061486100615861110280610861032
:1000500006118611492006108614061186154320C4
:10006000231C3628061086100611861523183C28F6
:1000700006108614061186114320061486100615F4
:100080008611A30110280530A2004920A20B4528A3
:100090000800A001A0034F20A00B4B280800A101DD
:0800A000A103A10B5128080087
:02400E00613F10
:00000001FF
